:100000000C943A000C9457000C9457000C94570031
:100010000C9457000C9457000C9457000C94570004
:100020000C9457000C9457000C9457000C945700F4
:100030000C9457000C9457000C9457000C945700E4
:100040000C9457000C9457000C9457000C945700D4
:100050000C9457000C9457000C9457000C945700C4
:100060000C9457000C9457000C9457000C945700B4
:100070000C94570011241FBECFEFD2E0DEBFCDBFDE
:1000800011E0A0E0B1E0EAE8F1E002C005900D92D5
:10009000A030B107D9F711E0A0E0B1E001C01D9296
:1000A000A230B107E1F70E9473000C94C4000C94D5
:1000B0000000CF93DF93CDB7DEB7E5E2F0E010822A
:1000C000E4E2F0E01082E8E2F0E01082E7E2F0E043
:1000D0001082EBE2F0E01082EAE2F0E080E180835F
:1000E000DF91CF910895CF93DF93CDB7DEB70E9414
:1000F0005900A895E4E5F0E087EF8083E0E6F0E0C2
:1001000088E18083E0E6F0E01082E2E6F0E0108231
:10011000ABE2B0E0EBE2F0E0808180618C9388E8B4
:1001200093E1909301018093000109C08091000147
:1001300090910101019790930101809300018091BA
:10014000000190910101009789F7ABE2B0E0EBE28A
:10015000F0E090818FEE89238C9388E893E190936F
:1001600001018093000109C080910001909101017B
:10017000019790930101809300018091000190917B
:0A0180000101009789F7C4CFFFCFFB
:00000001FF
